:100000000C9471000C9499000C9499000C94990034
:100010000C9499000C9499000C9499000C949900FC
:100020000C9499000C9499000C9499000C949900EC
:100030000C9499000C9499000C9499000C949900DC
:100040000C9492010C9499000C9499000C949900D2
:100050000C9499000C9499000C9499000C949900BC
:100060000C9499000C94990005A84CCDB2D44EB9CB
:100070003836A9020C50B9918688083CA6AAAA2A4B
:10008000BE000000803F0000000023002600290081
:1000900000000000240027002A00000000002500C6
:1000A00028002B00040404040404040402020202D5
:1000B000020203030303030301020408102040802B
:1000C00001020408102001020408102000000008AA
:1000D000000201000003040700000000000000000F
:1000E000A80411241FBECFEFD8E0DEBFCDBF11E0C2
:1000F000A0E0B1E0E0EAFFE002C005900D92A2307E
:10010000B107D9F721E0A2E0B1E001C01D92A3320E
:10011000B207E1F710E0C1E7D0E004C02197FE018B
:100120000E94C807C037D107C9F70E94DC010C94B0
:10013000CE070C940000833081F028F4813099F0D0
:100140008230A9F008958730A9F08830C9F0843052
:10015000B1F4809180008F7D03C0809180008F7703
:1001600080938000089584B58F7784BD089584B509
:100170008F7DFBCF8091B0008F778093B000089582
:100180008091B0008F7DF9CF1F93CF93DF93282FFD
:1001900030E0F901E453FF4F8491F901E854FF4F37
:1001A000D491F901EC55FF4FC491CC23A9F0162F3F
:1001B00081110E949B00EC2FF0E0EE0FFF1FE6562E
:1001C000FF4FA591B4918FB7F894EC91111108C02D
:1001D000D095DE23DC938FBFDF91CF911F910895DF
:1001E000DE2BF8CFCF93DF9390E0FC01E854FF4F74
:1001F00024918C559F4FFC0184918823D1F090E08D
:10020000880F991FFC01E057FF4FA591B491FC01A5
:10021000E656FF4FC591D491623071F49FB7F894C0
:100220003C91822F809583238C93E8812E2B288309
:100230009FBFDF91CF9108958FB7F894EC912E2B4B
:100240002C938FBFF6CF1F93CF93DF93182FEB0123
:1002500061E00E94F200209739F460E0812FDF9185
:10026000CF911F910C94C400CF3FD10511F461E0F0
:10027000F5CFE12FF0E0E453FF4FE491E33031F1AB
:1002800040F4E130B1F0E230E1F0C038D1057CF764
:10029000E4CFE73029F1E83059F1E430B1F780914B
:1002A0008000806280938000D0938B00C0938A008E
:1002B00004C084B5806884BDC7BDDF91CF911F9114
:1002C000089584B5806284BDC8BDF7CF8091800059
:1002D000806880938000D0938900C0938800EDCF20
:1002E0008091B00080688093B000C093B300E5CFE8
:1002F0008091B00080628093B000C093B400DDCFE5
:100300008E50806480937C0080917A00806480931A
:100310007A0080917A0086FDFCCF809178009091E0
:10032000790008951F920F920FB60F9211242F9308
:100330003F938F939F93AF93BF9380911F019091B1
:100340002001A0912101B091220130911E0123E0F2
:10035000230F2D3758F50196A11DB11D20931E01C5
:1003600080931F0190932001A0932101B09322015B
:1003700080911A0190911B01A0911C01B0911D0167
:100380000196A11DB11D80931A0190931B01A093AA
:100390001C01B0931D01BF91AF919F918F913F912F
:1003A0002F910F900FBE0F901F90189526E8230FE6
:1003B0000296A11DB11DD2CF789484B5826084BD10
:1003C00084B5816084BD85B5826085BD85B5816059
:1003D00085BD80916E00816080936E0010928100D7
:1003E0008091810082608093810080918100816092
:1003F0008093810080918000816080938000809153
:10040000B10084608093B1008091B00081608093DE
:10041000B00080917A00846080937A0080917A00A5
:10042000826080937A0080917A00816080937A0064
:1004300080917A00806880937A001092C10062E017
:1004400084E00E94F20061E083E00E94F20061E03B
:100450008BE00E94F20090E080E00E94BC0490E0FB
:1004600090930101809300018130910541F00A973A
:1004700031F081E090E0909301018093000183E2EC
:100480008093B00081E08093B10082E88093800087
:1004900089E1809381008FEF90E0909387008093B3
:1004A0008600E0E0AE2EE0E0BE2E8FB7F894C0905C
:1004B0001F01D0902001E0902101F09022018FBF18
:1004C000C0921601D0921701E0921801F092190122
:1004D000E0EDF0E08491ECEBF0E0C491E8EAF0E0CC
:1004E000D491DD2379F081110E949B00ED2FF0E083
:1004F000EE0FFF1FEA57FF4FA591B4918C91C823CF
:1005000081E009F480E0109214011092150190919D
:100510001301891751F080931301C0920E01D092FC
:100520000F01E0921001F092110180910E01909163
:100530000F01A0911001B0911101C81AD90AEA0A5D
:10054000FB0A80910A0190910B01A0910C01B091DE
:100550000D018C159D05AE05BF05B0F490911201FB
:1005600080911301981781F080931201911103C0BB
:1005700021E0813009F020E020931401913009F44A
:10058000811190E09093150180911501882381F0ED
:10059000809100019091010161E0019709F46AE006
:1005A000609300011092010190E080E00E94C40479
:1005B0008EE00E948001EC0181E10E948001AC018B
:1005C000CE01DD0FAA0BBB0B052E000C660B770BC3
:1005D000840F951FA61FB71FD0E0C0E0B7FD08C06D
:1005E000EC0181159440A105B10514F0CFEFD3E0E3
:1005F0008FE00E9480018C0182E10E948001012E27
:10060000000C220B330B092E000CAA0BBB0B800F26
:10061000911FA21FB31F10E000E0B7FD08C08C01BE
:1006200081159440A105B10514F00FEF13E080E1AE
:100630000E9480011C0183E10E9480014C014090D6
:100640001601509017016090180170901901809167
:10065000060190910701A0910801B0910901481687
:1006600059066A067B0609F461C1B801110F880BAF
:10067000990B0E94EE0520E030EC4FE754E40E9415
:1006800044056B017C014092060150920701609283
:100690000801709209012DE033E34CEC5DE30E9408
:1006A0003F0510E018166CF52AE836E24AE95EE3E9
:1006B000C701B6010E943F0511E0181614F528E2A3
:1006C00030EA40E05FE3C701B6010E943F0512E057
:1006D0001816BCF42BE03DE244E35FE3C701B6012A
:1006E0000E943F0513E0181664F42EEE39EB47E63E
:1006F0005FE3C701B6010E943F0515E018160CF034
:1007000014E0BE01DD0F880B990B0E94EE0520E07E
:1007100030EC4FE754E40E94440520E030EC4FE712
:1007200054E40E94A30626EA3BE944EC5AE30E9403
:10073000A3066B017C016091000170910101072EFD
:10074000000C880B990B0E94EE059B01AC01C701C0
:10075000B6010E94A3062AE037ED43E25CE30E9463
:10076000D30420E030E04AE75FE30E94A3062FE6CF
:1007700032E143E85AE30E94A3062091020130913E
:10078000030140910401509105010E94D3046B01C3
:100790007C0120E030E040E85FE30E949E0687FF96
:1007A0001FC0C0920201D0920301E0920401F092B6
:1007B0000501609102017091030180910401909103
:1007C0000501123009F446C0E0F4112321F1113083
:1007D00069F1C12CD12C50E8E52E5FE3F52E48C01D
:1007E00020E030E040E85FE3C701B6010E94D20498
:1007F00060930201709303018093040190930501BB
:10080000D8CF133009F499C0143019F79B01AC010B
:100810000E94D30418C02BED3FE049EC50E40E9445
:10082000A3060E9410076B017C0122C020E030E08B
:1008300040E05FE30E94D2049F7720E030E040E890
:1008400050E40E94A3069B01AC0160E070E080E8E8
:100850009FE37BC020E030E040E05FE30E943F0583
:10086000C12CD12C60E8E62E6FEBF62E87FDB1CFC0
:10087000B10137FE02C06D5F7F4F75956795759525
:100880006795C40197FC03969595879595958795EF
:10089000680F791F6F3F710519F014F06FEF70E06A
:1008A000072E000C880B990B0E94EE0520E030E02B
:1008B0004FE753E40E944405A70196010E94A30656
:1008C00020E030E040E05FE30E94A30620E030E05B
:1008D00040E05FE30E94D30420E030E04FE753E4C0
:1008E0000E94A30620E030E040E05FE30E94D304D2
:1008F0000E94B605EB016F3F710519F014F0CFEFC0
:10090000D0E0D7FF02C0D0E0C0E0BE018BE00E9483
:100910002301CE0126E0880F991F2A95E1F76FEF9A
:1009200070E00E94A00783E00E942301A114B1049B
:1009300009F4BBCD0E940000B4CD9B01AC010E9424
:10094000D30420E030E040E85FE30E94D2046BCFA4
:10095000EAE0F1E082E390E0A0E0B0E08083918300
:10096000A283B383148215821682178281E0808766
:100970008187128613860895F999FECF92BD81BDB5
:10098000F89A992780B50895262FF999FECF1FBAB6
:1009900092BD81BD20BD0FB6F894FA9AF99A0FBEA8
:1009A000019608955058BB27AA270E94EA040C9488
:1009B00064060E94560638F00E945D0620F039F465
:1009C0009F3F19F426F40C9453060EF4E095E7FBD0
:1009D0000C944D06E92F0E94750658F3BA1762076A
:1009E00073078407950720F079F4A6F50C94970611
:1009F0000EF4E0950B2EBA2FA02D0B01B90190013A
:100A00000C01CA01A0011124FF27591B99F0593F7D
:100A100050F4503E68F11A16F040A22F232F342FC5
:100A20004427585FF3CF469537952795A795F04013
:100A30005395C9F77EF41F16BA0B620B730B840B28
:100A4000BAF09150A1F0FF0FBB1F661F771F881FE0
:100A5000C2F70EC0BA0F621F731F841F48F4879538
:100A600077956795B795F7959E3F08F0B0CF93952A
:100A7000880F08F09927EE0F9795879508950E94A3
:100A8000290608F481E008950E9458050C94640634
:100A90000E945D0658F00E94560640F029F45F3F20
:100AA00029F00C944D0651110C9498060C945306A1
:100AB0000E94750668F39923B1F3552391F3951BB2
:100AC000550BBB27AA2762177307840738F09F5F6F
:100AD0005F4F220F331F441FAA1FA9F335D00E2EDC
:100AE0003AF0E0E832D091505040E695001CCAF749
:100AF0002BD0FE2F29D0660F771F881FBB1F26170C
:100B000037074807AB07B0E809F0BB0B802DBF01E2
:100B1000FF2793585F4F3AF09E3F510578F00C94B1
:100B20004D060C9498065F3FE4F3983ED4F3869507
:100B300077956795B795F7959F5FC9F7880F911DD2
:100B40009695879597F90895E1E0660F771F881FBE
:100B5000BB1F621773078407BA0720F0621B730B71
:100B6000840BBA0BEE1F88F7E09508950E94BD052F
:100B70006894B1110C94980608950E947D0688F03F
:100B80009F5798F0B92F9927B751B0F0E1F0660F51
:100B9000771F881F991F1AF0BA95C9F714C0B13092
:100BA00091F00E949706B1E008950C949706672F84
:100BB000782F8827B85F39F0B93FCCF386957795C1
:100BC0006795B395D9F73EF49095809570956195AA
:100BD0007F4F8F4F9F4F0895E89409C097FB3EF4D5
:100BE00090958095709561957F4F8F4F9F4F99237A
:100BF000A9F0F92F96E9BB279395F69587957795F8
:100C00006795B795F111F8CFFAF4BB0F11F460FFB7
:100C10001BC06F5F7F4F8F4F9F4F16C0882311F00F
:100C200096E911C0772321F09EE8872F762F05C023
:100C3000662371F096E8862F70E060E02AF09A95BE
:100C4000660F771F881FDAF7880F9695879597F9B3
:100C50000895990F0008550FAA0BE0E8FEEF16164D
:100C60001706E807F907C0F012161306E407F507A0
:100C700098F0621B730B840B950B39F40A2661F014
:100C8000232B242B252B21F408950A2609F4A140B7
:100C9000A6958FEF811D811D089597F99F6780E8C4
:100CA00070E060E008959FEF80EC089500240A94BE
:100CB0001616170618060906089500240A94121637
:100CC0001306140605060895092E0394000C11F46A
:100CD000882352F0BB0F40F4BF2B11F460FF04C017
:100CE0006F5F7F4F8F4F9F4F089557FD9058440F70
:100CF000551F59F05F3F71F04795880F97FB991F7B
:100D000061F09F3F79F08795089512161306140637
:100D1000551FF2CF4695F1DF08C0161617061806C4
:100D2000991FF1CF86957105610508940895E8949F
:100D3000BB2766277727CB0197F908950E942906DC
:100D400008F48FEF08950E94B6060C9464060E9482
:100D5000560638F00E945D0620F0952311F00C94A1
:100D60004D060C94530611240C9498060E947506A7
:100D700070F3959FC1F3950F50E0551F629FF001EE
:100D8000729FBB27F00DB11D639FAA27F00DB11D07
:100D9000AA1F649F6627B00DA11D661F829F222790
:100DA000B00DA11D621F739FB00DA11D621F839F17
:100DB000A00D611D221F749F3327A00D611D231FED
:100DC000849F600D211D822F762F6A2F11249F573B
:100DD00050409AF0F1F088234AF0EE0FFF1FBB1F3E
:100DE000661F771F881F91505040A9F79E3F5105FD
:100DF00080F00C944D060C9498065F3FE4F3983E07
:100E0000D4F3869577956795B795F795E7959F5FA6
:100E1000C1F7FE2B880F911D9695879597F9089538
:100E20009F930E941A070F9007FCEE5F0C944307F4
:100E30000C9453060E947D06D8F3E894E0E0BB27AB
:100E40009F57F0F02AED3FE049EC06C0EE0FBB0FD4
:100E5000661F771F881F28F0B23A6207730784075E
:100E600028F0B25A620B730B840BE3959A9572F7D4
:100E7000803830F49A95BB0F661F771F881FD2F712
:100E800090480C945907EF93E0FF07C0A2EA2AEDBF
:100E90003FE049EC5FEB0E94EA040E9464060F9079
:100EA000039401FC9058E8E6F0E00C9465079F3F3E
:100EB00031F0915020F4879577956795B795880F15
:100EC000911D9695879597F908959F938F937F939A
:100ED0006F93FF93EF939B01AC010E94A306EF91E8
:100EE000FF910E9479072F913F914F915F910C9450
:100EF000A306DF93CF931F930F93FF92EF92DF929E
:100F00007B018C01689406C0DA2EEF010E94B606C0
:100F1000FE01E894A5912591359145915591A6F34F
:100F2000EF010E94EA04FE019701A801DA9469F733
:100F3000DF90EF90FF900F911F91CF91DF91089577
:100F400097FB072E16F4009407D077FD09D00E9476
:100F5000B40707FC05D03EF4909581959F4F089506
:100F6000709561957F4F0895AA1BBB1B51E107C087
:100F7000AA1FBB1FA617B70710F0A61BB70B881F29
:100F8000991F5A95A9F780959095BC01CD010895B8
:100F9000EE0FFF1F0590F491E02D0994F894FFCF18
:020FA00001004E
:00000001FF
